:100000000C9472000C949A000C949A000C949A0030
:100010000C949A000C949A000C949A000C949A00F8
:100020000C949A000C949A000C949A000C949A00E8
:100030000C949A000C949A000C949A000C949A00D8
:100040000C9407050C949A000C949A000C949A0056
:100050000C949A000C949A000C949A000C949A00B8
:100060000C949A000C949A000000000023002600D3
:100070002900005EBCE2613FDD83C29C7E20A3FDBF
:100080001F41009D23BE46DB65F88C11AF32CA5775
:10009000E97400000000240027002A00000000008E
:1000A000250028002B0004040404040404040202B4
:1000B00002020202030303030303010204081020E7
:1000C00040800102040810200102040810200000F2
:1000D0000008000201000003040700000000000007
:1000E0000000040811241FBECFEFD8E0DEBFCDBF53
:1000F00011E0A0E0B1E0E0E1F5E102C005900D9271
:10010000A033B107D9F721E0A0E3B1E001C01D920F
:10011000A337B207E1F710E0C2E7D0E004C02197AF
:10012000FE010E94800AC137D107C9F70E9451051C
:100130000C9469080C94000090E0FC01E253FF4F1E
:100140002491FC01E654FF4F3491FC01EA55FF4F26
:10015000E491EE23C9F0222339F0233001F1A8F411
:10016000213019F1223029F1F0E0EE0FFF1FE456A3
:10017000FF4FA591B4918FB7F894EC91611126C00F
:1001800030953E233C938FBF08952730A9F0283047
:10019000C9F0243049F7809180008F7D03C08091A1
:1001A00080008F7780938000DFCF84B58F7784BD08
:1001B000DBCF84B58F7DFBCF8091B0008F778093AC
:1001C000B000D2CF8091B0008F7DF9CF3E2BDACF37
:1001D000CF93DF9390E0FC01E654FF4F24918A55C2
:1001E0009F4FFC0184918823D1F090E0880F991FE4
:1001F000FC01EE56FF4FA591B491FC01E456FF4F70
:10020000C591D49161110EC09FB7F8948C91E22FE3
:10021000E0958E238C932881E223E8839FBFDF91B2
:10022000CF9108958FB7F894EC91E22BEC938FBFA8
:10023000F6CF3FB7F8948091430190914401A0918B
:100240004501B091460126B5A89B05C02F3F19F086
:100250000196A11DB11D3FBFBA2FA92F982F882746
:10026000BC01CD01620F711D811D911D43E0660F20
:10027000771F881F991F4A95D1F70895DC0180E008
:10028000615090F09D919827E92FEF70F0E0EE58C3
:10029000FF4F2491E92FE295EF70F0E0EE57FF4F0A
:1002A000E491822F8E27ECCF0895DC012C911196DA
:1002B000ED91FC91F8948181822B81839281322F80
:1002C00030959323928382E090E00197F1F781814A
:1002D0008323818380E190E00197F1F79081789406
:1002E000E6E6F0E03197F1F7922381E009F480E04F
:1002F0000895FC0190810180F281E02D292F209545
:1003000060FF14C0F8948281822382838181892BCB
:100310008183A0E1B0E01197F1F78281982B92835D
:1003200078948AE690E00197F1F70895F894828135
:10033000822382838181892B8183AEE7B0E011978C
:10034000F1F78281982B9283789486E090E0EBCF4E
:10035000DF92EF92FF920F931F93CF93DF93EC0105
:10036000D62EE42E08E010E0FF24F39461E08D2DFA
:100370008F2109F460E0CE010E947901FF0C015049
:100380001109A1F7E11010C0F894E981FA81918177
:100390008881809589238183E981FA81928188818E
:1003A0008095892382837894DF91CF911F910F915B
:1003B000FF90EF90DF900895EF92FF920F931F93BD
:1003C000CF93DF938C017B0140E065E50E94A8019B
:1003D000E70188E0E80EF11C699140E0C8010E9445
:1003E000A801CE15DF05C1F7DF91CF911F910F91C5
:1003F000FF90EF900895AF92BF92CF92DF92EF926D
:10040000FF920F931F93CF93DF936C017B018B01BE
:10041000040F151FEB015E01AE18BF08C017D1070E
:1004200059F06991D601ED91FC910190F081E02D98
:10043000C6010995892B79F7C501DF91CF911F91ED
:100440000F91FF90EF90DF90CF90BF90AF90089505
:10045000089590E080E00895FC0190810180F28190
:10046000E02DF8948181292F20958223818378942F
:100470003DE7315011F180818923D9F3F8948281CD
:10048000822382838181892B81837894ACEBB3E0D2
:100490001197F1F7F894818182238183A8E8B0E075
:1004A0001197F1F78081982381E009F080E078943A
:1004B000E0E3F3E03197F1F7089580E00895AF921B
:1004C000BF92CF92DF92EF92FF920F931F93CF9341
:1004D000DF938B01BC0180914D0190914E010E94F0
:1004E000DC0140E06EEB80914D0190914E010E9445
:1004F000A801E801680189E0C80ED11CA0904D0157
:10050000B0904E0188E0E82EF12C10E001E0C5012A
:100510000E9455018111102B000F81E0E81AF108AB
:10052000B1F71993CC16DD0649F780914D019091F2
:100530004E010E942C0291E0813009F090E0892F59
:10054000DF91CF911F910F91FF90EF90DF90CF90AF
:10055000BF90AF9008950F931F93CF93DF93CDB7C4
:10056000DEB729970FB6F894DEBF0FBECDBF8C0162
:1005700080914D0190914E010E942C02811102C088
:1005800080E01FC0BE016F5F7F4FC8010E945F0205
:100590008823B1F368E0CE0101960E943E0199855F
:1005A0008913EECF8D818F33B9F020F48F3141F76D
:1005B00089E007C08F3521F08F3711F78CE001C03B
:1005C0008BE029960FB6F894DEBF0FBECDBFDF914A
:1005D000CF911F910F9108958AE0F3CFBF92CF92F0
:1005E000DF92EF92FF920F931F93CF93DF93EC0173
:1005F000B62EC72E8D85811105C0CE010E942C021A
:1006000081110EC01B861D861C8680E0DF91CF9174
:100610001F910F91FF90EF90DF90CF90BF900895C2
:1006200040E060EFCE010E94A80101E0E12CD12C56
:1006300011E0CE010E945501F82ECE010E94550115
:1006400091E0F91218C0813099F51134D8F2DB86A7
:10065000D11002C081E08D878B81882399F2239687
:10066000EB2DFC2DCF01089629912193E817F9076E
:10067000D9F781E0CBCFEE2DF0E0F8120FC08B85DB
:100680001817A0F4DE01AE0FBF1F13968C918023C4
:1006900079F4F12C193008F41C87D12EEC0FFD1FD2
:1006A0008381902F9095892383830AC08113F1CF92
:1006B000FE01EE0DF11D8381802B8383FF24F394D3
:1006C0006F2DCE010E9479011F5F000F11F4E3949A
:1006D00001E087E08E1508F0ACCFB7CFCF93DF9362
:1006E000EC0160E08E810E949C0061E08E810E949E
:1006F0009C0060E08E810E949C0084EC90E0019759
:10070000F1F7DF91CF910895CF92DF92EF92FF92B0
:100710000F931F93CF93DF936C017C0187E0E80E6A
:10072000F11CD0E0C0E0062F10E0B8010C2E02C092
:10073000759567950A94E2F76170F70181917F01E1
:100740000E949C002196C430D10579F7C601DF9143
:10075000CF911F910F91FF90EF90DF90CF900C946D
:100760006E03CF92DF92EF92FF920F931F93CF937E
:10077000DF93EC01F62E642F8C810E949C008D810A
:100780008F3F19F060E00E949C000F2D10E08F85D4
:1007900084FF25C06E0187E0C80ED11CF12CE12C2E
:1007A000B8010E2C02C0759567950A94E2F7617046
:1007B000F60181916F010E949C00FFEFEF1AFF0A82
:1007C00088E0E816F10461F7CE01DF91CF911F9127
:1007D0000F91FF90EF90DF90CF900C946E03B801D3
:1007E00084E0759567958A95E1F7CE010E948403B0
:1007F0006F2DCE01DF91CF911F910F91FF90EF9060
:10080000DF90CF900C94840340E0682F8BE591E05B
:100810000C94B103CF93DF93823029F490916A0155
:10082000986090936A0180936E0110926F0180E44A
:100830008093700180E18093710180E58093720163
:1008400061E080915F010E94E800809160018F3F2C
:1008500019F061E00E94E80061E0809161010E946E
:10086000E800CBE5D1E09E012B55314080916A0133
:1008700084FD0BC084E090E021962817390744F4EA
:1008800061E08E810E94E800EECF88E090E0F4CF36
:100890008CE996E80197F1F760E080915F010E9492
:1008A0009C0060E0809161010E949C008091600149
:1008B0008F3F19F060E00E949C0080916A0184FDE6
:1008C00039C063E08BE591E00E948403C4E2D3E287
:1008D000CE010197F1F763E08BE591E00E9484037C
:1008E0002197F1F763E08BE591E00E94840388E2B1
:1008F00091E00197F1F762E08BE591E00E948403BB
:1009000080916A0180620E94040484E080936B01FC
:100910008CE00E94040481E00E9404048CE99FE0C2
:100920000197F1F782E080936C0186E0DF91CF912F
:100930000C94040480620E94040484E293E2019710
:10094000F1F780916A0180620E94040488E291E0DC
:100950000197F1F780916A0180620E940404D0CF70
:1009600041E00E94B10381E090E00895FC01019014
:100970000020E9F73197AF01481B590BBC018BE50B
:1009800091E00C94FB018F929F92AF92BF920F93D4
:100990001F93CF93DF93CDB7DEB7A1970FB6F8942F
:1009A000DEBF0FBECDBF19A2423008F44AE08E016F
:1009B0000F5D1F4F842E912CB12CA12CA501940109
:1009C0000E944A0AE62FB901CA01EA30F4F4E05D58
:1009D000D801EE938D01232B242B252B79F790E062
:1009E00080E0109719F0CD010E94B604A1960FB6D1
:1009F000F894DEBF0FBECDBFDF91CF911F910F9155
:100A0000BF90AF909F908F900895E95CE1CF1F92C7
:100A10000F920FB60F9211242F933F938F939F93B2
:100A2000AF93BF9380913F0190914001A09141010C
:100A3000B091420130913E0126E0230F2D3758F549
:100A40000296A11DB11D20933E0180933F0190931A
:100A50004001A0934101B0934201809143019091E4
:100A60004401A0914501B09146010196A11DB11D1F
:100A70008093430190934401A0934501B0934601B4
:100A8000BF91AF919F918F913F912F910F900FBE8A
:100A90000F901F90189529E8230F0396A11DB11DF3
:100AA000D2CFCF93DF93CDB7DEB761970FB6F8946F
:100AB000DEBF0FBECDBF789484B5826084BD84B59F
:100AC000816084BD85B5826085BD85B5816085BD49
:100AD00080916E00816080936E0010928100809101
:100AE0008100826080938100809181008160809389
:100AF0008100809180008160809380008091B100AE
:100B000084608093B1008091B00081608093B000D8
:100B100080917A00846080937A0080917A0082606C
:100B200080937A0080917A008E7F80937A00809102
:100B30007A00806880937A001092C10082E00E945F
:100B40000A04E1E080916E018111E0E0E195F0E0BE
:100B5000E55AFE4F848980680E94040482E191E096
:100B60000E94B604E0914D01F0914E011386158666
:100B700014861286118610861782168215821482B8
:100B8000138210924B0110924C0101E0BE016F5F85
:100B90007F4F80914D0190914E010E94EE0288237B
:100BA00009F468C067E0CE0101960E943E01988575
:100BB0008913ECCF80914701811128C080914D01AC
:100BC00090914E010E942C02BE016F5F7F4F809179
:100BD0004D0190914E010E94DC0140E064EB809158
:100BE0004D0190914E010E94A80180914D0190917C
:100BF0004E010E945501182F80914D0190914E0198
:100C00000E942C02111102C000934701109148016B
:100C10008981803109F4F4C1CE0101960E94AB02B2
:100C20008117C0F4809148018093480180914B0165
:100C30008F5F80934B018981883231F0A8F4803135
:100C400019F0823209F0A2CF80914C018F5F80931E
:100C50004C019CCF8981803111F48CE0E5CFCE012D
:100C600001960E94AB02E0CF8B3371F3823409F01E
:100C70008DCFEACF00E010E080914D0190914E01C0
:100C80000E942C0240E06CEC80914D0190914E014D
:100C90000E94A8014091470164E480914D01909128
:100CA0004E010E94A80180914901882309F444C0A3
:100CB000E0914801E950FEEECF2EF2E0DF2EE33066
:100CC00038F4F0E0EE0FFF1FE45FFE4FC080D180EC
:100CD00080914A01882309F488C0809147018111DD
:100CE00084C08FB7F89480903F0190904001A0900D
:100CF0004101B09042018FBF0D2C000CEE08FF089F
:100D000080914D0190914E010E9455018130A1F0DA
:100D10002FB7F89480913F0190914001A09141013B
:100D2000B09142012FBF8C199D09AE09BF098815EA
:100D30009905AA05BB0520F3E0916E01E23008F0A9
:100D40007EC0E150F0E0E55AFE4F848980680E9441
:100D50000404E0914D01F0914E011386158614862E
:100D600012861186108617821682158214821382CB
:100D7000BE01665F7F4F80914D0190914E010E94B0
:100D8000EE02882381F067E0CE010A960E943E01C0
:100D90009989891308C080914D0190914E010E945C
:100DA0002C0281114EC0C12CD12C8EEFE82E82EC8A
:100DB000F82E46015701E894B7F82FEF3FEF4FE7C1
:100DC0005FE7C501B4010E94310A8111A0C02FEF75
:100DD0003FEF4FE75FE7C501B4010E94D90818163D
:100DE0000CF095C086E291E085C00D2C000CEE0859
:100DF000FF080E9419014B015C01C114D104E104F8
:100E0000F10489F499CF21E0C21AD108E108F10870
:100E100048EE840E43E0941EA11CB11CC114D10401
:100E2000E104F10451F30E941901681979098A0952
:100E30009B09683E73408105910528F7DECFE1E00C
:100E400081CFBE016F5F7F4FCE010A960E945F0285
:100E5000882309F4A8CF68E0CE0101960E943E01E4
:100E600099858913A0CF6A8170E0762F6627770F66
:100E7000770F770F298188E0289F90011124262B76
:100E8000372B8A858031D1F4688570E08F81AB0182
:100E9000481B5109CA019695982F882797958795E1
:100EA0000E94360ACB014097B90153E0660F771FC5
:100EB0005A95E1F760789C01260F371F213854EED0
:100EC00035070CF470CFB901330F880B990B0E94D2
:100ED0000F0920E030E040E05CE30E94C4096B01B0
:100EE0007C01AC019B010E94310A882309F461CF87
:100EF00082E291E00E94B6048EE291E00E94B60484
:100F00000115110509F4B8CE0E940000B5CE2FEFEF
:100F10003FEF4FE75FE4C701B6010E94BF09181613
:100F20001CF48AE291E0E6CF2FEF3FEF4FE75FEC52
:100F3000C701B6010E94D90887FDF3CF20E030E059
:100F4000A901C701B6010E94D90887FF0AC041E084
:100F50006DE28BE591E00E94B103F7FAF094F7F8A7
:100F6000F0942AE037ED43EA5BE3C701B6010E9443
:100F70006D084B015C010E94DE086B017C010E9440
:100F80000D099B01AC01C501B4010E946C084B0125
:100F90005C014AE0C701B6010E94C30441E06EE271
:100FA0008BE591E00E94B10320E030E040E251E4A3
:100FB000C501B4010E94C4094B015C010E94DE0816
:100FC0006B01F12CE12C4AE0C701B6010E94C30479
:100FD000C701B6010E940D099B01AC01C501B40116
:100FE0000E946C0820E030E040E251E40E94C40915
:100FF0000E94DE0890E080E04AE00E94C3047CCFBB
:101000001D3008F00FCE29CE60E08BE00E94E80092
:10101000E5ECF0E0E491A0E3B1E0EC93E1EBF0E08B
:10102000E491F0E0EE0FFF1FE859FF4F8591949196
:1010300012969C938E9311971B961C921B971D964C
:101040001C921D971C961C921C971A961C921A971C
:1010500019961C92199718961C92189717961C921D
:10106000179716961C92169715961C92159714961C
:101070001C92149713961C921397E7E4F1E0B78340
:10108000A68314821582108289E0818381E08283A5
:101090008383138A128AEBE5F1E01382128284E0E3
:1010A00091E09183808387E084838FEF858386E05E
:1010B000868382E0878383E0808784E0818785E080
:1010C00082871386148615861686178681E00C940F
:1010D0000A04F8940C94860A5058BB27AA270E9449
:1010E00084080C9485090E94770938F00E947E09D3
:1010F00020F039F49F3F19F426F40C9474090EF48F
:10110000E095E7FB0C946E09E92F0E94960958F3CD
:10111000BA17620773078407950720F079F4A6F5DC
:101120000C94B8090EF4E0950B2EBA2FA02D0B01EC
:10113000B90190010C01CA01A0011124FF27591B1C
:1011400099F0593F50F4503E68F11A16F040A22F22
:10115000232F342F4427585FF3CF46953795279593
:10116000A795F0405395C9F77EF41F16BA0B620B92
:10117000730B840BBAF09150A1F0FF0FBB1F661FD9
:10118000771F881FC2F70EC0BA0F621F731F841F1C
:1011900048F4879577956795B795F7959E3F08F042
:1011A000B0CF9395880F08F09927EE0F9795879504
:1011B00008950E944A0908F481E008950E949E095A
:1011C00088F09F5798F0B92F9927B751B0F0E1F008
:1011D000660F771F881F991F1AF0BA95C9F714C0B8
:1011E000B13091F00E94B809B1E008950C94B809AB
:1011F000672F782F8827B85F39F0B93FCCF38695F1
:1012000077956795B395D9F73EF49095809570954D
:1012100061957F4F8F4F9F4F0895E89409C097FBCA
:101220003EF490958095709561957F4F8F4F9F4FBD
:101230009923A9F0F92F96E9BB279395F695879501
:1012400077956795B795F111F8CFFAF4BB0F11F4C4
:1012500060FF1BC06F5F7F4F8F4F9F4F16C088236B
:1012600011F096E911C0772321F09EE8872F762FA1
:1012700005C0662371F096E8862F70E060E02AF0E2
:101280009A95660F771F881FDAF7880F96958795CE
:1012900097F90895990F0008550FAA0BE0E8FEEFA3
:1012A00016161706E807F907C0F012161306E4072A
:1012B000F50798F0621B730B840B950B39F40A2623
:1012C00061F0232B242B252B21F408950A2609F401
:1012D000A140A6958FEF811D811D089597F99F6705
:1012E00080E870E060E008959FEF80EC08950024AE
:1012F0000A941616170618060906089500240A947B
:1013000012161306140605060895092E0394000C00
:1013100011F4882352F0BB0F40F4BF2B11F460FF8F
:1013200004C06F5F7F4F8F4F9F4F089557FD9058B8
:10133000440F551F59F05F3F71F04795880F97FB99
:10134000991F61F09F3F79F0879508951216130653
:101350001406551FF2CF4695F1DF08C01616170682
:101360001806991FF1CF86957105610508940895B7
:10137000E894BB2766277727CB0197F908950E9449
:101380004A0908F48FEF08950E94D7090C94850943
:101390000E94770938F00E947E0920F0952311F011
:1013A0000C946E090C94740911240C94B9090E94D0
:1013B000960970F3959FC1F3950F50E0551F629FFA
:1013C000F001729FBB27F00DB11D639FAA27F00D9E
:1013D000B11DAA1F649F6627B00DA11D661F829FC5
:1013E0002227B00DA11D621F739FB00DA11D621FAA
:1013F000839FA00D611D221F749F3327A00D611DC7
:10140000231F849F600D211D822F762F6A2F1124A8
:101410009F5750409AF0F1F088234AF0EE0FFF1FDB
:10142000BB1F661F771F881F91505040A9F79E3F32
:10143000510580F00C946E090C94B9095F3FE4F3F8
:10144000983ED4F3869577956795B795F795E79588
:101450009F5FC1F7FE2B880F911D9695879597F991
:1014600008950E944A09880B990B089597FB072E4F
:1014700016F4009407D077FD09D00E946C0A07FC8F
:1014800005D03EF4909581959F4F08957095619594
:101490007F4F0895A1E21A2EAA1BBB1BFD010DC0B0
:1014A000AA1FBB1FEE1FFF1FA217B307E407F50714
:1014B00020F0A21BB30BE40BF50B661F771F881FF0
:1014C000991F1A9469F760957095809590959B0186
:1014D000AC01BD01CF010895AA1BBB1B51E107C0A0
:1014E000AA1FBB1FA617B70710F0A61BB70B881FB4
:1014F000991F5A95A9F780959095BC01CD01089543
:10150000EE0FFF1F0590F491E02D0994F894FFCFA2
:1015100000000000B004FB01290228025E00BC00AC
:1015200077012040456C656374726F50657070651B
:1015300072006E616E00696E66006F766600430031
:00000001FF
